:020000040000FA
:020000001128C5
:08000800A300030E8312A40003
:10001000A00A0319A10A0B11240E8300A30E230EBC
:10002000090083167F3086008312861383163F30C3
:1000300092008312003095009701971517158316CB
:1000400086118312121092101215831681128111DB
:100050000115811401148312A001A1012210203086
:1000600095008617D4208613D4208617D4208613B3
:10007000D4208617D420861300309500D420D420B5
:10008000D420D4200618502886185228061A592839
:10009000861A5B2822184D284228061F622842280B
:1000A00022144228D420861C422895202218652834
:1000B0006F2895206F28D420D420D420B320B320DB
:1000C000B3204228952022106F282214861C6B280A
:1000D000061F6D286528AC20422822106F28810158
:1000E000CD2086187E28061A8228861A84280618AB
:1000F0008C280530210203199128712806186520E3
:10010000A1017128A1017128D120A620A101D4202C
:10011000B320B320B3204228D120AC202214A10167
:100120004228D120A620A1014228950AD82040309B
:100130001502031D95288617080004309507D8205E
:1001400040301502031D9D28861708009503D8200E
:10015000031DA6288613080004309502D820031D2D
:10016000AC28861308009501861340309500861749
:10017000D820D82095018613D82004309507D820A0
:1001800020301502031DBD288617D82004309502A3
:10019000D820031DC628861308000B118B168B1759
:1001A00008008B128B130800FA30A600E02008002C
:1001B0003230A600E02008000130A600E020080050
:1001C000F930A7000000000000000000000000005F
:1001D000000000000000000000000000000000001F
:1001E000000000000000A70BE228A60BE028080092
:02400E00423F2F
:104200004B0046005A002D0049006E006E0065000C
:104210006E006C006900630068007400640069004F
:104220006D006D0065007200200028004300290029
:10423000200032003000300033002000620079009E
:10424000200043006F006F006C00430068006900AD
:024250007000FC
:00000001FF
